:020000040000FA
:10000000000000008031A628230091002300950104
:1000100015141308910A0319920A200008002300FE
:1000200093000430950055309600AA309600951440
:100030009518FE331511910A0319920A2000080041
:10004000A801A700FF30A707031CA807031C08008E
:100050000330A400DF302E20F533A401E83EA300D6
:10006000A409FC30031C0332A3070318FD33A307C4
:100070000000A40FF93323180032A31C0232000041
:1000800000320800B201B301B401B5012130A9006A
:100090002032B20DB30DB40DB50D2B0832022C0871
:1000A000031C2C0F33022D08031C2D0F34022E08C5
:1000B000031C2E0F3502031C0C32B5002B08B202B4
:1000C0002C08031C2C0FB3022D08031C2D0FB402A7
:1000D0000314A30DA40DA50DA60DA90BDA33350845
:1000E000AE003408AD003308AC003208AB000800A5
:1000F000AC01AB011030AF00240DAB0DAC0D2708E7
:10010000AB022808AC3B031805322708AB072808C8
:10011000AC3D0310A30DA40DAF0BEE332308080074
:100120001030B100A401A301B00CAF0C031C0432C9
:100130002708A3072808A43DA40CA30CAC0CAB0C07
:10014000B10BF2332B0808002000080023008C01BB
:10015000220091016A3021009900980120008C0151
:1001600022008C010B3021008C00951324008C00A0
:1001700023008C0120008C180A326430803120204A
:100180008C1805328C180132FD33843134240C1262
:100190008C120C11003080310420BD00803106200B
:1001A000BE00063080310420BB0080310620BC0038
:1001B000083080310420DC00093080310420DD006B
:1001C000023080310420E000CC16601CCC124C16AA
:1001D000E01C4C12CC17601DCC13D614E01DD610B9
:1001E0004C17601E4C135616E01E5612D616601F92
:1001F000D612D613A6010F30A5004230A40040301D
:10020000A3003B08AB003C08AC00AD01AE0180315F
:1002100042202408B8002308B7003836BA00370C4B
:10022000B900A6011230A5004F30A4008030A30011
:100230003D08AB003E08AC00AD01AE01803142206C
:100240002608C4002508C3002408C2002308C100F2
:100250000430A400B030A3003E08A8003D08A70069
:1002600080317820C5002408C6004408A600430851
:10027000A5004208A4004108A3003708AB003808D5
:10028000AC00AD01AE01803142202408C800230833
:10029000C7008831561AF22801300C180030B60019
:1002A00001308C190030B604031902328431F8246D
:1002B0000C11D61385318C1C012DD61A0E328431C7
:1002C000DC24013056190030B6000130D619003058
:1002D000B60403190132033201326E32E9334C1A8B
:1002E0000232033201321132E3338431DC245619F5
:1002F000033256148231AA228431DC24D619033207
:100300005614823124225610D3334C10CC10843131
:10031000DC24003056190130B6000030D619013007
:10032000B604031901320E324C1D063256148231C6
:10033000AA228231242205325614823124228231AB
:10034000AA22E3334C10CC108431DC24D6190332BA
:100350005614823124228431DC244C1C033256147E
:100360008231AA228431DC24013056190030B600D3
:100370000130D6190030B60503190132C633843175
:10038000DC245619033256148231AA22CC1C0332C3
:100390005614823124224C10CC108431DC240030DD
:1003A00056190130B6000030D6190130B6050319D0
:1003B000023256107D33A9330C08DF005F08A3001A
:1003C0005E08890AA30C890BFD330130031C003041
:1003D000013903195613031D5617561B693356145A
:1003E000561B2632CC1F01320C16CC1E0432561C72
:1003F00002328C160C153A08A400390880312E20E0
:100400000C123A08A400390880312E200C08DF00B5
:100410005F08A3005E08890AA30C890BFD33013035
:10042000031C0030013903195613031D5617D83326
:10043000CC1E01328C12323080312020CC1E013291
:100440000C115610813158294C150C150A30803189
:100450002020CA01C901490847024A08483B031C39
:100460005E32CC1F01320C16D61F04323C30803174
:100470002D203F32013056180030B6000030D6181B
:100480000130B60503190732CC1A03320C118C1255
:1004900002320C158C16013056180030B6000130AF
:1004A000D6180030B605031902320C118C12003038
:1004B00056180130B6000130D6180030B6050319C1
:1004C0000732CC1A03320C118C1202320C158C1626
:1004D000003056180130B6000030D6180130B6058D
:1004E00003190732CC1A03320C118C1202320C158C
:1004F0008C163A08A400390880312E200C123A08D4
:10050000A400390880312E208431DC2456190132B0
:100510004C140130C9070030CA3D031C9C33D61F60
:1005200006324608A8004508803121200800CC1E6C
:1005300001328C124636A800450CA70080312220DB
:10054000CC1E01320C114636A800450CA7008031A4
:10055000222008004C110C150A3080312020480858
:10056000B0004708AF00A8010330A70080319020F9
:10057000A1002C08A200CA01C901490821024A08A9
:10058000223B031C5E32CC1F01320C16D61F0432F4
:100590003C3080312D203F32013056180030B600FB
:1005A0000030D6180130B60503190732CC1A0332D1
:1005B0000C118C1202320C158C16013056180030BA
:1005C000B6000130D6180030B605031902320C11FE
:1005D0008C12003056180130B6000130D6180030A9
:1005E000B60503190732CC1A03320C118C120232F1
:1005F0000C158C16003056180130B6000030D61895
:100600000130B60503190732CC1A03320C118C12D3
:1006100002320C158C163A08A400390880312E20BD
:100620000C123A08A400390880312E208431DC24D1
:10063000D6190132CC140130C9070030CA3D031C61
:100640009C33D61F06324608A80045088031212079
:100650000800CC1E01328C124636A800450CA700BB
:1006600080312220CC1E01320C114636A800450CE8
:10067000A7008031222008000330D0000530CF00D1
:100680008331AB2308000330D0000730CF00833123
:10069000AB2308000430D0000230CF008331AB23FD
:1006A00008000230D000CF008331AB2308000230B5
:1006B000D0000130CF008331AB2308000430D000DC
:1006C0000E30CF008331AB2308000230D000CF00C2
:1006D0008331AB234608B0004508AF00A8010330C2
:1006E000A70080319020A7002C08A800803122208C
:1006F0000330D000CF018331AB2308000130D0009C
:10070000CF008331AB234608B0004508AF00A801F5
:100710000330A70080319020A7002C08A80080316A
:1007200022200230D000CF008331AB234608B00036
:100730004508AF00A8010330A70080319020A70032
:100740002C08A800803122200330D0000630CF00D2
:100750008331AB230800D1015114501C5110D11426
:10076000D01CD1105115501D5111D103CB01CB011B
:100770004B085102031C1D325008A4004F08A3006F
:100780004B08890AA40CA30C890BFC330130031C11
:100790000030D200D208031D02328231AA22013079
:1007A0005202031D0232823124220130CB07031C86
:1007B000DF330800CA01C901D101CC11D001CF013A
:1007C0008431DC2456191332CC155108A301A4013D
:1007D000890A0314A30DA40D890BFC332408FF3AE6
:1007E000D0052308FF3ACF058231AA22D10A8431ED
:1007F000DC24D6191132CC155108A301A401890AB1
:100800000314A30DA40D890BFC332408D004230882
:10081000CF0482312422D10ACA01C90107304A0219
:10082000031C0632031D1D32D13049020318193250
:1008300001302000803120208431DC240130561921
:100840000030B6000130D6190030B6040319033267
:10085000CA01C901B5330130C9070030CA3D031CC4
:10086000DD335108D0000800BE011230BD00CC16A7
:100870004C16CC17D6100230BC00BC30BB00DC01DB
:100880000430DD005612D6122300910120003D08ED
:1008900080310F203E0880310F2006302300910068
:1008A00020003B0880310F203C0880310F200830A9
:1008B0002300910020005C0880310F2009302300C4
:1008C000910020005D0880310F206014CC1E601064
:1008D000E0144C1EE0106015CC1F6011E015D61C12
:1008E000E01160164C1F6012E016561EE0126017F1
:1008F000D61E601302302300910020006008803172
:100900000F2087310F270330D0000530CF0083310F
:10091000AB234608B0004508AF00A8010330A7008C
:1009200080319020A7002C08A800803122200130BF
:10093000D000CF008331AB234608B0004508AF009C
:10094000A8010330A70080319020A7002C08A80040
:10095000803122200330D0000730CF008331AB2319
:100960004608B0004508AF00A8010330A700803159
:100970009020A7002C08A800803122200130D00050
:10098000CF008331AB234608B0004508AF00A80173
:100990000330A70080319020A7002C08A8008031E8
:1009A00022200130D000CF018331AB230330A800D7
:1009B000E8308031212008004C1B0D3283108C1947
:1009C000831483185615831C56110C0C0318D61566
:1009D000031CD6110C320C0C03185615031C5611AF
:1009E00083108C1983148318D615831CD611080024
:1009F0000C1802320330DE008C190132DE01D616EB
:100A00000800323080312020D61E0A323230803148
:100A100020208C180132FD330A30D7008831F228AB
:100A20000832CE08031D053250304D028831031CB8
:100A3000F2282000CA01C9018C1839328431DC2423
:100A4000013056190030B6000130D6190030B60416
:100A5000031919320330A80020308031212084315D
:100A6000DC24013056190030B6000130D6190030B0
:100A7000B605031902328831FB288831561DF52846
:100A80008831D61DF8280A3080312020C90A031980
:100A9000CA0ACA08031D0432C9304902031C0632BF
:100AA00020000C15D61783313C230632C533490884
:100AB000CD004A08CE00B5338331DA23CC19043295
:100AC00083316523813158294F03023003195006C1
:100AD000031D2232CC1F103283315123CC136015F9
:100AE000CC1F60110230230091002000600880318B
:100AF0000F20813158291032CC1783314A23CC176B
:100B00006015CC1F601102302300910020006008A6
:100B100080310F20813158295008043A0E300319D2
:100B20004F06031D043283313C238731ED275008E3
:100B3000043A0A3003194F06031D043283313C2363
:100B400088310C205008033A063003194F06031D64
:100B50002132561E1032833151235612E016561E92
:100B6000E0120230230091002000600880310F2045
:100B7000813158290F3283314A235616E016561E0A
:100B8000E0120230230091002000600880310F2025
:100B9000813158294F03013003195006031D0432D7
:100BA00083313C238631E02E5008043A0B30031980
:100BB0004F06031D043283313C238731BC2F50087C
:100BC000033A023003194F06031D21324C1E103226
:100BD000833157234C12E0144C1EE01002302300E6
:100BE00091002000600880310F20813158290F3298
:100BF00083315E234C16E0144C1EE01002302300BB
:100C000091002000600880310F2081315829500860
:100C1000043A0D3003194F06031D2132CC1E103249
:100C200083315123CC126014CC1E6010023023009B
:100C300091002000600880310F20813158290F3247
:100C400083314A23CC166014CC1E6010023023007E
:100C500091002000600880310F2081315829500810
:100C6000043A093003194F06031D1F3283313C2318
:100C70004C1F0E324C1360164C1F601202302300C2
:100C800091002000600880310F20813158290D32F9
:100C90004C1760164C1F6012023023009100200098
:100CA000600880310F20813158295008033A0530FF
:100CB00003194F06031D043283313C238831482831
:100CC0005008033A073003194F06031D03328331DE
:100CD0003C231F3250034F04031D173283313C2342
:100CE0008C168431DC24561901328C12D61901324B
:100CF0008C168C1809328C126430803120208C18AC
:100D00000132FD3381315829EC3383316523813140
:100D100058298331DA23CC19043283316523813198
:100D20005829873163270A305302031C0432833168
:100D300065238131582982312422B0015308AF0044
:100D4000A8010A30A70080319020D4008331DA2333
:100D5000CC190432833165238131582987316327C7
:100D60000A305302031C0432833165238131582930
:100D70005308D50054085507BD00BE01BE0D3D08FF
:100D80003E04031D0332BE010130BD00BE08031D39
:100D900004322E303D02031C04322000BE012D30EF
:100DA000BD002300910120003D0880310F203E0846
:100DB00080310F2087310F2783313C23813158291F
:100DC0008431DC24561907328231AA22BD0A031964
:100DD000BE0A87310F278431DC24D61908328231CC
:100DE000AA220130BD020030BE3B87310F278C188C
:100DF00015323230803120202300910120003D083F
:100E000080310F203E0880310F208C180132FD33D5
:100E100087310F2783313C2381315829D133A601F3
:100E20000F30A5004230A4004030A3003B08AB00C7
:100E30003C08AC00AD01AE01803142202408B8006E
:100E40002308B7003836BA00370CB900A6011230B3
:100E5000A5004F30A4008030A3003D08AB003E0841
:100E6000AC00AD01AE01803142202608C400250847
:100E7000C3002408C2002308C1000430A400B0301D
:100E8000A3003E08A8003D08A70080317820C500D7
:100E90002408C6004408A6004308A5004208A40090
:100EA0004108A3003708AB003808AC00AD01AE0123
:100EB000803142202408C8002308C700080083317D
:100EC0003C23813158290A30D3005008053A4F0499
:100ED000031D0132D3014F03053003195006031DD2
:100EE00002320130D3005008053A033003194F068F
:100EF000031D02320230D3005008053A07300319AF
:100F00004F06031D02320330D3005008053A0F305C
:100F100003194F06031D02320430D3005008053A6E
:100F20001F3003194F06031D02320530D30050084D
:100F3000053A1E3003194F06031D02320630D30056
:100F40005008053A1C3003194F06031D02320730C2
:100F5000D3005008053A183003194F06031D02321A
:100F60000830D3005008053A103003194F06031D0E
:100F700002320930D30008008431DC2456190832CB
:100F80000A30BB070030BC3D87310F278231AA22CF
:100F90008431DC24D61908320A30BB020030BC3B55
:100FA00087310F278231AA228C18163232308031D5
:100FB000202006302300910020003B0880310F20C4
:100FC0003C0880310F208C180132FD3387310F2708
:100FD00083313C2381315829CF338331DA23CC1933
:100FE00004328331652381315829873163270530E5
:100FF0005302031C0432833165238131582953087D
:10100000DC0008302300910020005C0880310F20B4
:1010100083313C23813158298331DA23CC190432BE
:101020008331652381315829873163270A30530280
:10103000031C0432833165238131582982312422F3
:10104000B0015308AF00A8010A30A70080319020FA
:10105000DD008331DA23CC190432833165238131F9
:101060005829873163270A305302031C0432833125
:101070006523813158295308DD0709302300910089
:1010800020005D0880310F2083313C2381315829B5
:101090008331DA23CC190432833165238131582915
:1010A0004F03053003195006031D05320A30DA00DC
:1010B0004630DB0028325008053A033003194F064A
:1010C000031D05324730DA008330DB001C32500844
:1010D000053A073003194F06031D05328430DA0044
:1010E000C130DB0010325008053A0F3003194F06AB
:1010F000031D0532C230DA00FE30DB0004328331DA
:1011000065238131582983313C235A08D700833124
:10111000DA23CC19483283314323C830D80057082A
:10112000230091002000580880310F20D70A57086B
:101130005B02031D0B32C930D800D70357082300C8
:1011400091002000580880310F204832CA01C9019F
:1011500007304A02031C0632031D1B32D1304902FC
:101160000318173220008431DC2401305619003076
:10117000B6000130D6190030B60403190132C73366
:101180000130803120200130C9070030CA3D031CE6
:10119000DF33C930D80057082300910020005808D9
:1011A00080310F201B32823124228931F2215708ED
:1011B000230091002000590880310F20D70A5708DA
:1011C0005B02031D0A32C930D80057082300910082
:1011D0002000580880310F200132993383317E235B
:1011E000813158290A30DA0008324730DA000532F6
:1011F0008430DA000232C230DA00561432308031E4
:101200002020D61A11328431DC24013056190030E6
:10121000B6000130D6190030B60403190332843108
:10122000DC24F3335A08D700D61A21328431DC2467
:10123000013056190030B6000130D6190030B6041E
:10124000031915323230803120208431DC24013002
:1012500056190030B6000130D6190030B604031913
:1012600003328431DC24F3335610813158298C1831
:1012700009323230803120208C180132FD33561073
:1012800081315829570880310420D900C8305902CB
:10129000031D10324608B0004508AF00A801073012
:1012A000A70080319020A7002C08A80080312220C0
:1012B000D70ABA33C9305902031D013214328B31B7
:1012C000CA238331AB234608B0004508AF00A8010C
:1012D0000330A70080319020A7002C08A80080319F
:1012E0002220D70AA133DC08031D033256108131B6
:1012F000582901305C020130031D0030B6000A306D
:101300005A020130031D0030B60503190132303294
:1013100002305C020130031D0030B60047305A0233
:101320000130031D0030B6050319013221320330AC
:101330005C020130031D0030B60084305A020130D7
:10134000031D0030B60503190132123204305C026D
:101350000130031D0030B600C2305A020130031DB7
:101360000030B60503190132033256108131582975
:10137000CA01C901CA08031D1C325D0849020318CD
:1013800018320330A800E830803121208431DC2479
:10139000013056190030B6000130D6190030B604BD
:1013A0000319013208328C1C0632C90A0319CA0A11
:1013B000E1338831FD283230803120208431DC2433
:1013C000013056190030B6000130D6190030B6048D
:1013D000031903328431DC24F3338C180132FD33DA
:1013E000813158294F03023003195006031D023280
:1013F0004130D9005008043A0E3003194F06031D3E
:1014000002324230D9005008043A0A3003194F061C
:10141000031D02324330D9005008033A0630031945
:101420004F06031D02324430D9004F030130031927
:101430005006031D02324530D9005008043A0B30E3
:1014400003194F06031D02324630D9005008033AF3
:10145000043003194F06031D02324730D9005008EB
:10146000043A0F3003194F06031D02324830D900E9
:101470005008023A033003194F06031D0232493067
:10148000D9004F03043003195006031D02324A30BD
:10149000D9005008033A023003194F06031D0232E7
:1014A0004B30D9005008043A0D3003194F06031D84
:1014B00002324C30D9005008023A4F04031D023268
:1014C0004D30D9005008023A023003194F06031D6F
:1014D00002324E30D9005008033A4F04031D023245
:1014E0004F30D9005008043A093003194F06031D44
:1014F00002325030D9005008043A043003194F0624
:10150000031D02325130D9005008033A0530031947
:101510004F06031D02325230D9005008033A0730FB
:1015200003194F06031D02325330D90050034F04F4
:10153000031D02325430D9005008033A0330031916
:101540004F06031D02325530D9005008043A0730C7
:1015500003194F06031D02325630D9004F030330E2
:1015600003195006031D02325730D9005008043ABF
:10157000063003194F06031D02325830D9005008B7
:10158000043A023003194F06031D02325930D900C4
:101590005008043A0C3003194F06031D02325A302A
:1015A000D9004F03053003195006031D02323130B4
:1015B000D9005008053A033003194F06031D0232C3
:1015C0003230D9005008053A073003194F06031D81
:1015D00002323330D9005008053A0F3003194F0654
:1015E000031D02323430D9005008053A1F30031968
:1015F0004F06031D02323530D9005008053A1E301F
:1016000003194F06031D02323630D9005008053A3F
:101610001C3003194F06031D02323730D900500821
:10162000053A183003194F06031D02323830D9002D
:101630005008053A103003194F06031D02323930A5
:10164000D9005008053A4F04031D02323030D9004A
:101650005008063A153003194F06031D02322E308A
:10166000D9005008063A0C3003194F06031D023208
:101670002C30D9005008063A333003194F06031DA9
:1016800002323F30D9005008063A0A3003194F069B
:10169000031D02322130D9005008063A38300319B0
:1016A0004F06031D02323A30D9005008063A2D3059
:1016B00003194F06031D02322230D9005008063AA2
:1016C000213003194F06031D0132D9015008053A94
:1016D0000E3003194F06031D02323D30D900500869
:1016E000053A163003194F06031D02322F30D90078
:1016F0005008053A123003194F06031D02322830F4
:10170000D9005008063A123003194F06031D023261
:101710002930D9005008053A1D3003194F06031D22
:1017200002322630D9005008063A2A3003194F06F3
:10173000031D02323B30D9005008053A1530031919
:101740004F06031D02322B30D9005008063A1E30D6
:1017500003194F06031D02322D30D9005008063AF6
:10176000133003194F06031D02325F30D9005008B1
:10177000073A373003194F06031D02322430D900CF
:101780005008063A293003194F06031D0232403033
:10179000D900080041305902031D04320230D00044
:1017A0000130CF0042305902031D04320430D00012
:1017B0000E30CF0043305902031D04320430D000F4
:1017C0000A30CF0044305902031D04320330D000E8
:1017D0000630CF0045305902031D03320130D000DE
:1017E000CF0046305902031D04320430D0000B30C4
:1017F000CF0047305902031D04320330D0000430BB
:10180000CF0048305902031D04320430D0000F309D
:10181000CF0049305902031D04320230D00003309A
:10182000CF004A305902031D04320430D000013089
:10183000CF004B305902031D04320330D000023078
:10184000CF004C305902031D04320430D0000D305B
:10185000CF004D305902031D03320230D000CF01BA
:101860004E305902031D03320230D000CF004F30FA
:101870005902031D03320330D000CF01503059020A
:10188000031D04320430D0000930CF00513059021A
:10189000031D03320430D000CF0052305902031D23
:1018A00004320330D0000530CF0053305902031DFD
:1018B00004320330D0000730CF0054305902031DEA
:1018C00003320130D000CF0155305902031D0332DD
:1018D0000330D000CF0056305902031D04320430CB
:1018E000D0000730CF0057305902031D04320330B7
:1018F000D0000130CF0058305902031D04320430AB
:10190000D0000630CF0059305902031D0432043094
:10191000D0000230CF005A305902031D0432043087
:10192000D0000C30CF0031305902031D0432053095
:10193000D0000130CF0032305902031D043205308F
:10194000D0000330CF0033305902031D043205307C
:10195000D0000730CF0034305902031D0432053067
:10196000D0000F30CF0035305902031D043205304E
:10197000D0001F30CF0036305902031D043205302D
:10198000D0001E30CF0037305902031D043205301D
:10199000D0001C30CF0038305902031D043205300E
:1019A000D0001830CF0039305902031D0432053001
:1019B000D0001030CF0030305902031D0332053003
:1019C000D000CF012E305902031D04320630D00062
:1019D0001530CF002C305902031D04320630D000E0
:1019E0000C30CF003F305902031D04320630D000C6
:1019F0003330CF0021305902031D04320630D000AD
:101A00000A30CF003A305902031D04320630D000AC
:101A10003830CF0022305902031D04320630D00086
:101A20002D30CF00D908031D04320630D0002130FC
:101A3000CF003D305902031D04320530D0000E3076
:101A4000CF002F305902031D04320530D00016306C
:101A5000CF0028305902031D04320530D000123067
:101A6000CF0029305902031D04320630D000123055
:101A7000CF0026305902031D04320530D0001D303E
:101A8000CF003B305902031D04320630D0002A300B
:101A9000CF002B305902031D04320530D000153021
:101AA000CF002D305902031D04320630D0001E3005
:101AB000CF005F305902031D04320630D0001330CE
:101AC000CF0024305902031D04320730D0003730D4
:101AD000CF0040305902031D04320630D0002930B7
:081AE000CF000800FF33FF33C3
:020000040001F9
:02000E00840963
:02001000FF1CD3
:00000001FF
